:020000040800F2
:10000000E0040020D900000805140008F9120008D7
:1000100000000000000000000000000000000000E0
:100020000000000000000000000000004F14000865
:1000300000000000000000004D14000851140008EA
:10004000EB000008EB000008EB000008EB000008E4
:10005000EB000008EB000008EB000008EB000008D4
:1000600000000000EB000008EB000008EB000008B7
:10007000EB000008EB00000800000000EB000008A7
:1000800000000000EB00000800000000000000007D
:10009000EB00000800000000EB000008EB00000887
:1000A000EB000008EB000008EB000008B5190008A1
:1000B000EB000008EB00000800000000000000005A
:1000C0000448854600F090F800480047FD190008F4
:1000D000C046C046E004002004488047044800476A
:1000E000FEE7FEE7FEE7FEE7FEE7FEE7C5140008D1
:1000F000C100000830B50B46014600202022012433
:1001000009E00D46D5409D4205D31D469540491B4B
:100110002546954040191546521E002DF1DC30BD94
:10012000F0B51FB40646002082B005464024019178
:1001300000901BE0019922460F46304600F042F83D
:10014000049A059B801A994110D3104619462246FD
:1001500000F028F8361A8F4101972246012000212D
:10016000009F00F01FF838184D4100902046641E93
:100170000028DFDC019B00982946324607B0F0BD1D
:10018000D2B201E00270401C491EFBD2704700222F
:10019000F6E710B513460A4604461946FFF7F0FF86
:1001A000204610BD10B5202A04DB0146203A9140BC
:1001B000002010BD914020239C1A0346E3401943C0
:1001C000904010BD10B5202A04DB0846203AD040EC
:1001D000002110BD0B46D340D0402024A21A9140EC
:1001E0000843194610BD0000064C0125064E05E0E7
:1001F000E36807CC2B430C3C98471034B442F7D348
:10020000FFF762FF481A0008681A0008704770B5C7
:100210000024014620314A79022A03D00421C16317
:10022000012418E0026813680E25AB4313600268CE
:1002300013685B085B001360436C1C2213400122AF
:1002400015469D40036C5D604A7100220A71816B06
:10025000002900D08847204670BD0000F8B5002373
:100260000124A2E027469F403A4070D04D68022DFD
:1002700001D0122D14D1DD08AD002D1800952D6A86
:100280005E07AC46F50E0F26AE46AE406546B5435A
:10029000AC460E697546AE4065462E43009D2E6203
:1002A0004D68012D05D0022D03D0112D01D0122D46
:1002B00016D185680326AC465D00AE46AE40654665
:1002C000B543AC46CE687546AE4065462E43866063
:1002D00046680D79BE43ED06ED0F9D403543456000
:1002E00006685F000325BD40AE46AE430D79B446B7
:1002F000AE07B60FBE4065462E430660C66875461B
:10030000AE438D68BD403543C5604D68ED004BD5AB
:10031000294D6E6B26436E639E08284DB6007519F5
:10032000AC46AD689E07360F0F27B740BD43052783
:100330003F07B84201D1002715E0214FB84201D153
:10034000012710E01F4FB84202D102270BE02BE03B
:100350001D4FB84201D1032705E01C4FB84201D11F
:10036000052700E00627B7402F436546AF60184DCC
:100370002E684F689643FF0300D516432E606E68C3
:100380004F689643BF0300D516436E60AE684F6852
:100390009643FF0200D51643AE60EE684F68964361
:1003A000BF0200D51643EE605B1C0A681546DD40AF
:1003B00000D057E7F8BD00000010024000000140E7
:1003C0000004005000080050000C0050001C0050B9
:1003D00000040140002A01D08161704781627047AA
:1003E00001480068704700000C00002070B502460C
:1003F00040325378202B1CD11378012B19D00123C4
:10040000137024245470046825689D432560046893
:1004100025681E03B5432560046825680D432560E3
:10042000006801681943016020205070002010709E
:1004300070BD022070BD70B5024640325378202B4B
:100440001BD11378012B18D001241470242353706E
:1004500003681D68A5431D6005682B680F263602DA
:10046000B343090219432960006801682143016010
:10047000202050700020107070BD022070BD000060
:1004800070B5040006D0254640356878002600285F
:1004900002D005E0012070BD2E70204600F04AF821
:1004A00024206870206801684908490001600F2114
:1004B0006068090688432168086121688A6801200C
:1004C000C00382438A60E1680129A16808D0212223
:1004D0009202114322689160E168022902D005E08E
:1004E0000143F7E701212268C902516021684A6887
:1004F0000F4B1A434A602168CA688243CA60616927
:1005000020690843A169090208432168C860216A7B
:10051000E0690843216808602068016801221143EE
:1005200001606664202068702663AE70002070BD94
:100530000080000210B586B0044614216846FFF71B
:1005400026FE1149206888421BD1104CE16A022026
:100550000143E162E16A01400320059180020090BD
:1005600012200190012002900320039006200490A5
:1005700069460748FFF772FEA06B01218905084311
:10058000A06306B010BD00000058004000100240FB
:100590000004005002480168491C016070470000D7
:1005A0000C00002010B508480024016840221143C7
:1005B0000160204600F00AF8002801D0012401E083
:1005C00000F01CF8204610BD0020024070B5054622
:1005D00009487D210024C9000068FFF78BFD00F069
:1005E000F9FB002801D0012404E000222946501E16
:1005F00000F01AF8204670BD100000200448416B3E
:10060000012211434163816B0204114381637047EE
:1006100000100240C106C90E01208840014908604F
:100620007047000000E100E010B500F0EDFE10BDE5
:10063000F8B504460078544D800672D5524E002716
:10064000403EB06BC00004D4B06BA9050843B06352
:1006500001274E480168C90511D40168821511436C
:100660000160FFF7BDFE009005E0FFF7B9FE0099BD
:10067000401A642837D845480068C005F5D5326867
:100680000321090560680A400140914208D08103B6
:10069000890F032904D13168890301D50120F8BDF0
:1006A0002A69032109040A4022D0084090421FD041
:1006B000207880061CD528692A6988430121C9044D
:1006C0000A432A612A698A432A612861C0050FD535
:1006D000FFF786FE009008E0FFF782FE0099411ABE
:1006E0002B48814201D90320F8BD28698005F3D544
:1006F00061688803800F032805D1326800058243B2
:1007000001400A43326028690322616812041140E3
:1007100008432861002F04D0B16B012000078143FA
:10072000B1632078C00705D0E868A1688008800020
:100730000843E8602078800705D5E8680C218843E5
:10074000E1680843E8602078400706D5E86803219F
:100750008902884321690843E8602078000706D5AC
:10076000E86803210903884361690843E860207849
:10077000000606D5E868032189048843A169084377
:10078000E8600020F8BD000040100240007000400A
:1007900088130000F8B50E4605007DD05348006868
:1007A000C007C00FB0420AD250480168490849004A
:1007B000314301600068C007C00FB04271D1287892
:1007C0004B4C800705D5E068F0218843A9680843B1
:1007D000E0602878C00752D06868022817D0032844
:1007E00018D02168012818D08905002959DAE16854
:1007F000890889000143E160FFF7F2FD6968074657
:10080000022912D003291CD0012926D033E0216807
:100810008903EAE721688901E7E74907E5E7FFF788
:10082000DFFDC11B3348814223D8E0680007800FF9
:100830000228F4D123E0FFF7D3FDC11B2D488142EC
:1008400017D8E0680007800F0328F4D117E0FFF7FE
:10085000C7FDC11B274881420BD8E0680007800F05
:100860000128F4D10BE0FFF7BBFDC11B21488142F9
:1008700001D90320F8BDE0680007800FF3D11B48C1
:100880000168C907C90FB1420DD90168490849007B
:1008900031430160006800E003E0C007C00FB042D0
:1008A00001D00120F8BD2878400706D5E06807216F
:1008B00009028843E9680843E0602878000707D503
:1008C000E0680721C90288432969C9000843E0603C
:1008D00000F036F8E168084A0906090F515CC84083
:1008E000064908600020FFF771FEF8BD00200240B5
:1008F0000010024088130000241A00081000002095
:10090000044805490068C968044A4905490F515C13
:10091000C840704710000020001002403D1A000837
:10092000044805490068C968044A8904490F515CB4
:10093000C840704710000020001002403D1A000817
:1009400010B5184AD1680C20084004280BD008289C
:1009500010D00C2810D050680004410F0120C003B3
:10096000491C884010BD1068C00601D50E4810BD56
:100970000E4810BD0E4810BD88020E4B000F185CCB
:100980000902D368890F491CDB0301D5084A05E039
:100990001268D20601D5044A00E0044A5043FFF72A
:1009A000A9FB10BD0010024000093D000024F40026
:1009B00000127A00341A0008FEB505007ED0FE4C05
:1009C000E7680C20E668074001200004064028780C
:1009D000C00747D0082F05D00C2F0AD101200004F2
:1009E000864206D1206880033CD568680028E5D09F
:1009F00038E0012069680004814203D12168014385
:100A0000216011E0052301221B0492049942216810
:100A100002D111432160F1E7814321602168014047
:100A20000091206890432060686800280DD0FFF78F
:100A3000D7FC009005E0FFF7D3FC0099401A64282A
:100A40007AD820688003F6D50CE0FFF7C9FC009047
:100A500005E0FFF7C5FC0099401A6428F0D820682B
:100A60008003F6D42878800755D50923E868042F39
:100A70000DD00C2F01D1002E09D000283BD02168C9
:100A8000994301432160FFF7ABFC064627E021684C
:100A9000490701D5002891D061681F2212029143B5
:100AA0002A69120211436160216899430143216060
:100AB000FFF746FFE16809060A0F00E079E1BF4948
:100AC000895CC840BE4908600020FFF77FFD002810
:100AD00072D120E0FFF784FC801B0228B0D8206888
:100AE0004007F7D560681F21090288432969090278
:100AF000084360600FE02068400840002060FFF776
:100B00006FFC064604E0FFF76BFC801B022897D8B9
:100B100020684007F7D42878C0065FD5002F0CD096
:100B2000A869002849D02068FF21013108432060CE
:100B3000FFF756FC06462DE0C0E02068800502D590
:100B4000A8690028A7D06068072149038843296A5B
:100B5000084360606068297F0002000A09060843B4
:100B60006060286A410B0120C003491C8840E1688D
:100B700009060A0F9149895CC84091490860002024
:100B8000FFF724FD002817D128E0FFF729FC801B80
:100B90000228A3D820688005F7D56068072149039B
:100BA0008843296A084360606068297F0002000A60
:100BB00009060843606011E0E1E02168FF20013090
:100BC00081432160FFF70CFC064604E0FFF708FCB8
:100BD000801B022872D820688005F7D42878794EC7
:100BE000000724D568690028306910D00121084326
:100BF0003061FFF7F5FB009005E0FFF7F1FB00998E
:100C0000401A02285AD830698007F6D50FE040080C
:100C100040003061FFF7E4FB009005E0FFF7E0FBE8
:100C20000099401A022849D830698007F6D42878FC
:100C3000400765D500200290A06BC00006D4A06BD1
:100C4000012109070843A063012002905E48016862
:100C5000C90511D40168821511430160FFF7C0FB7B
:100C6000009005E0FFF7BCFB0099401A642825D8E6
:100C700055480068C005F5D5FF20AA6801308242BA
:100C800003D131690143316111E001218902002A58
:100C900007D005231B029A4203D132690A4332610D
:100CA000EFE7326982433261306988433061A86876
:100CB00000280FD0FFF794FB009007E05EE0FFF7FD
:100CC0008FFB0099411A4148814257D8306980050D
:100CD000F5D50DE0FFF784FB009006E0FFF780FB01
:100CE0000099411A3948814248D830698005F5D4C5
:100CF0000298002804D0A06B012109078843A06353
:100D0000686A002864D00C2F3ED0012636060228DF
:100D1000206805D0B0432060FFF762FB05462FE056
:100D2000B0432060FFF75CFB074604E0FFF758FB89
:100D3000C01B022822D820688001F7D4E96AA86A7B
:100D4000E2680843296BFD231B049A4311430843BF
:100D5000E060206830432060FFF742FB054604E076
:100D6000FFF73EFB401B022808D820688001F7D51A
:100D70002EE0FFF735FB401B022801D90320FEBD02
:100D800020688001F5D423E00128F8D0E068012133
:100D90000904AA6A014091420BD10F218904EA6A31
:100DA0000140914205D1032189050840296B884201
:100DB0000ED00120FEBD000000100240241A0008E1
:100DC0001000002040100240007000408813000016
:100DD0000020EFE7094910B5401E884201D90120E3
:100DE00010BD074C60610321081F00F00DFB0020BF
:100DF000A06107202061002010BD0000FFFFFF0060
:100E000000E000E070477047F8B502680446D0691A
:100E10001168936805072D0F5BD0DD07ED0FFF26E6
:100E200021360E402E4367D0C60706D0CE0504D526
:100E300001261662E26F3243E26787070222042628
:100E4000002F06DADF0704D027683A62E76F3743DE
:100E5000E767470706D5DB0704D023681E62E36F08
:100E60001343E367020709D520220A402A4305D02D
:100E7000236808221A62E36F1343E367E26F002AD4
:100E80002FD0800606D5880604D5216E002901D012
:100E900020468847E06F21688968490601D4000729
:100EA00024D5204600F0D8FB20688168490619D572
:100EB0008168402291438160E06E002812D0204971
:100EC0008163E06EFFF7A3F900280AD0E06E816B22
:100ED00006E0850610D58D060ED5216E1CE0204655
:100EE0008847F8BD2046FFF78EFFF8BD2046FFF784
:100EF0008AFF0020E067F8BDC50208D55B0206D571
:100F00000120000510622046FFF77CFFF8BD0306B4
:100F100005D50B0603D5616E0029E0D1F8BD40066A
:100F2000FCD54806FAD51368204640218B43136050
:100F3000202161670021616600F0DDF9F8BD000045
:100F40004516000810B5040003D0606F002802D0D9
:100F500007E0012010BD002170200155204600F05F
:100F600027F824206067206801684908490001606B
:100F7000204600F0D9FB0128ECD0606A002802D09E
:100F8000204600F0C9FA206841680922D202914344
:100F90004160206881682A2291438160206801684D
:100FA000012211430160204600F01CFB10BD00002F
:100FB00010B586B0044614216846FFF7E8F81549D5
:100FC0002068884224D11448416B012292031143C6
:100FD0004163C16A01221143C162C06A694610407F
:100FE0000590032040020090022001900020029012
:100FF000032003900420049005200007FFF72EF93A
:10100000002211461B20FFF70FFB1B20FFF702FBFE
:1010100006B010BD0038014000100240F0B5836FEB
:10102000202B54D100290AD0002A08D08568DC0181
:10103000A54206D10369002B03D1CB0701D00120C3
:10104000F0BD034660331E7C012E40D001261E7485
:101050004165014640310A834A830022FF26026629
:10106000A54204D10569002D13D11A4D0AE07F274E
:10107000002D09D001263607B5420CD10569002D97
:1010800005D03F258D8307E00569002D01D08F83B2
:1010900002E08E8300E08A83C267222181670168B3
:1010A0008D68012635438D608168A14202D10169B6
:1010B00000290AD0084901661A7400680168FF22F5
:1010C0002132114301600020F0BD0449F3E7022002
:1010D000F0BD0000FF010000D116000879160008DD
:1010E00070B54E4CE078032806D032230522611FEC
:1010F0004B4800F099F870BD20794A4D012815D170
:101100006079012804D1012210212846FFF762F9F5
:101110006079002804D1002210212846FFF75AF9EF
:10112000322307223D493E4800F07EF8207902280C
:1011300015D16079012804D1012220212846FFF72A
:1011400049F96079002804D1002220212846FFF7C0
:1011500041F9322307223149314800F065F82079FE
:10116000032815D16079012804D1012240212846A5
:10117000FFF730F96079002804D100224021284689
:10118000FFF728F9322307222449254800F04CF8BC
:101190002079002823D1607901280ED10122102165
:1011A0002846FFF717F9012220212846FFF712F9F8
:1011B000012240212846FFF70DF9607900280ED161
:1011C000002210212846FFF705F900222021284699
:1011D000FFF700F9002240212846FFF7FBF82079AD
:1011E000042888D16079012809D1012210212846DC
:1011F000FFF7F0F8012220212846FFF7EBF860798D
:101200000028EED1002210212846FFF7E3F8002243
:1012100020212846FFF7DEF870BD00000500002001
:101220006000002000040050FFB50446406F83B00A
:1012300017460D4620285CD1002D0AD0002F08D07B
:10124000A168C001814207D12069002804D1E807C4
:1012500002D0012007B0F0BD204660300290007C33
:10126000012846D00298012101740020E067212066
:101270006067FFF7B5F826464036019037827782DF
:101280000120A1680003814202D12069002802D018
:101290002F46002511E000270FE000228021204684
:1012A00000F056FB002815D1002F15D021683878A2
:1012B00088627F1C708A401E7082708A019B0028A1
:1012C00006980090E9D100224021204600F040FB22
:1012D000002808D00320BDE728882168C005C00D7C
:1012E0008862AD1CE6E72020606702990020087440
:1012F000B0E70220AEE77047FEE70000F0B587B028
:1013000014216846FEF743FF1848C26A02210A43C7
:10131000C262C26A0A400592C16A01252943C162BC
:10132000C06A032428400526E402360705900022FF
:1013300021463046FFF74EF80D4F01227021384606
:10134000FFF748F80094002401950294694630465E
:101350000394FEF783FF7020009002946946019584
:1013600003943846FEF77AFF07B0F0BD0010024044
:101370000004005010B5144812490160E121C90071
:101380004160002181600161416181610122C1618F
:10139000C2600162FFF774F8002801D0FEF736FF43
:1013A00000210948FFF722F8002801D0FEF72EFFA0
:1013B00000210548FFF73FF8002801D0FEF726FF7F
:1013C00010BD0000005800401400002010B50C486B
:1013D0000A490160E1214902416000218160C16048
:1013E00001618161C1610C22016242614162FFF7CA
:1013F000A9FD002801D0FEF709FF10BD003801400B
:1014000060000020704700008307FF22DB0E9A4037
:101410008907090E994000280BDA0007000F0838E9
:10142000830808489B001818C36993430B43C361A2
:101430007047830804489B001B18186890430843B2
:101440001860704700ED00E000E400E0704770476E
:1014500010B5FFF79FF810BD30B599B0342168463C
:10146000FEF795FE14210DA8FEF791FE1C2112A88F
:10147000FEF78DFE124801680322D2029143C21486
:1014800089180160102000900520002440030125E8
:1014900008900695079409946846FFF78DFA0F2087
:1014A0000D900E940F941094002111940DA8FFF745
:1014B00071F912A812951494FFF7BAF819B030BD5B
:1014C0000070004010480168821511430160C16836
:1014D0000E4A1140C16001680D4A114001608168E7
:1014E000490849008160016801229204914301602A
:1014F000C168FD2212049143C160002101610549C8
:10150000C003886070470000001002400C40FF8854
:10151000F6FFF6FE00ED00E010B5818CC90707D09C
:1015200001684A6801235B049A43836A1A434A604C
:10153000818C890707D501684A6801231B049A43F7
:10154000C36A1A434A60818C490707D501684A6813
:1015500001239B049A43036B1A434A60818C090759
:1015600007D501684A680123DB039A43436B1A439A
:101570004A60818CC90607D50268916801231B0364
:101580009943836B19439160818C890607D5016863
:101590008A6801235B039A43C36B1A438A60818C78
:1015A000490612D503685A6801210905046C8A436B
:1015B00022435A60026C8A4207D1026851680323B1
:1015C0005B059943436C19435160818C090607D52B
:1015D00001684A680123DB04806C9A4302434A6035
:1015E00010BD0000F8B500260446C667FEF7F8FEF9
:1015F000054620680068124F000709D501212B46D7
:10160000002249052046009700F0A2F900280DD1DC
:101610002068006840070BD501212B460022890570
:101620002046009700F094F9002801D00320F8BD6F
:1016300020206067A067603426740020F8BD000099
:10164000FFFFFF0110B5806A0022014640314A8346
:101650004A82FFF7D8FB10BD01680A68FF232133D7
:101660009A430A6001688A68520852008A60202101
:10167000816700210166704710B5014640318B8BB0
:10168000846F0268222C04D090690821084390617D
:1016900010BD526A446D1A402280426D921C426510
:1016A0004A8B521E4A83498B0029F1D101680A688E
:1016B000FF2321339A430A6001688A685208520066
:1016C0008A602021816700210166FFF709FD10BDB6
:1016D00010B5014640318B8B846F0268222C04D0F8
:1016E000906908210843906110BD526A1A40436D09
:1016F0001A70426D521C42654A8B521E4A83498BB6
:101700000029F1D101680A68FF2321339A430A6056
:1017100001688A68520852008A602021816700218E
:101720000166FFF7DDFC10BDF8B504462669A26826
:10173000E76932436669102000253E43236832433F
:1017400078491E68784F3E4016431E6023685A68E9
:1017500003263603B243E66832435A602368A2691F
:101760008B4201D0266A32439E680B273F02BE435C
:1017700016439E606D4E23686D4AB3420CD1D26809
:101780009207920F06D0012A38D0022A34D0032AB9
:1017900020D11EE001201DE0664EB3420AD1D2687E
:1017A0000C26324026D0042A28D0082A24D00C2A1D
:1017B00010D10EE08B420DD1D66803229202164062
:1017C00018D001229202B61A18D0B61A14D0964236
:1017D00000D10820564A0126403A574FF6038B4263
:1017E00036D100280CD002280DD0042812D00828A9
:1017F0001FD11CE00020EDE70220EBE70420E9E721
:10180000FFF77EF808E01068C00601D5384605E00D
:101810004A4803E0FFF794F8002873D0626851004B
:101820005118814205D81103814202D303E03046AA
:10183000F4E7012566E0010E060250080023301887
:101840005941FEF76DFC03210902411A3C4A55E05B
:10185000E169B14232D1030000F0B4F809070A0D82
:1018600006250606062B0600E3E7FFF749F81CE00D
:10187000FFF756F819E010686168C00602D54808FD
:10188000304A01E0304A48088018FEF733FC80B245
:1018900001462E4A10399142CBD8511C0140000715
:1018A000400F08432CE0FFF74BF8616840004A08FE
:1018B000EAE76168012248081204E5E7030000F046
:1018C00081F809070A0D06260606062C0600B0E771
:1018D000FFF716F81DE0FFF723F81AE010686168BB
:1018E000C00602D54808C01902E014484A0810187A
:1018F000FEF700FC80B20146144A1039914298D894
:101900002168C8600020206660662846F8BDFFF7A1
:1019100017F861684A088018EAE761684808801982
:10192000E6E7000000480040F369FFEF003801409F
:10193000401002400044004000093D000024F40033
:10194000FFFC0F0000127A000048E801EFFF0000E2
:10195000FFB581B017460E4604460A9D09E0681C93
:1019600007D0FEF73DFD0499401AA8420CD8002D7F
:101970000AD02068C1693046884318D00020B84298
:10198000EDD0002005B0F0BD20680168FF22A13233
:1019900091430160206881684908490081602020E6
:1019A0006067A0670020603420740320EAE701200C
:1019B000E5E7000010B50248FFF726FA10BD000069
:1019C0006000002030B47446641E2578641CAB426D
:1019D00000D21D46635D5B00E31830BC184702E08F
:1019E00008C8121F08C1002AFAD1704770470020AA
:1019F00001E001C1121F002AFBD17047FEF7D2FDA2
:101A0000FFF72AFDFFF77AFCFFF7B4FCFFF7DEFCD7
:101A1000072202490248FFF701FBF9E70500002011
:101A2000600000200000000000000000010203042C
:101A300006070809030406080C10182030000000EF
:101A40000001020304000000681A000800000020E2
:101A500014000000DE1900087C1A000814000020A1
:101A6000CC040000EE190008FF0102030D00000085
:0C1A70000000000000000000000020004A
:04000005080000C12E
:00000001FF
